:03000000021143A7
:03000B000200A54B
:03002B000202AB23
:03005B0002040993
:030073000203E3A2
:1000800002030406080C10182030406080040608A3
:100090000C10182030406080A0C00D0D0405060D26
:1000A0000502030302C2AFC0D0C0E020620C20688A
:1000B00002419A306602415AE47385258AC262E59C
:1000C00025F470022121206802210E758B00D0E0FA
:1000D000D0D0C286C291C295D2AF32C286C291C27E
:1000E00095741AD5E0FDE53C1420E21520E10D20C1
:1000F0007D02D296307D02D29002011ED292020180
:100100001E207D02D290307D02D29602011E758B98
:1001100000D0E0D0D0C286C291C295D2AF32758BEA
:1001200000D0E0D0D0D2AF32419AE525600A207DE0
:1001300002D286307D02D295C291419AE5256002B5
:10014000D291207D02C295307D02C286419AE5257A
:10015000600A207D02D295307D02D286207D02C2C7
:1001600086307D02C295419A207D02C290307D0288
:10017000C296207D02C296307D02C290740ED5E0F8
:10018000FDE525600A207D02D286307D02D295C22F
:1001900091419A207D02C290307D02C296C2927433
:1001A0000ED5E0FDE525600A207D02D286307D0275
:1001B000D295C291419AC292207D02C290307D02B6
:1001C000C296740ED5E0FDE5256002D291207D0235
:1001D000C295307D02C286419AC292207D02C296AB
:1001E000307D02C290740ED5E0FDE5256002D2910B
:1001F000207D02C295307D02C286419A207D02C2D6
:1002000096307D02C290C292740ED5E0FDE5256065
:100210000A207D02D295307D02D286207D02C286E0
:10022000307D02C295419A207D02C296307D02C285
:1002300090207D02C290307D02C296740ED5E0FD02
:10024000E525600A207D02D295307D02D286207D90
:1002500002C286307D02C295419A30723DE53C2053
:10026000E21A20E129207D02C290307D02C2962050
:100270007D02C296307D02C29002029A20E1E62001
:100280007D02C290307D02C296C29202029AC29250
:10029000207D02C296307D02C290E525F4F58A7574
:1002A0008B00D262D0E0D0D0D2AF32C2AFC2AD5359
:1002B000E6EFC0D0C0E0D2D3D2AFC2CEE52960070E
:1002C0002074461529610978007900E580307E01A7
:1002D000F430E50278FF53DACF207E0343DA203092
:1002E0007E0343DA10C2D8C271E580307E01F4305B
:1002F000E50279FFC3E89970CE30610375291820B3
:1003000074037529188859D270E52A6004152A618A
:100310001920740543DA01C2D82070026180A859FF
:10032000206102C2702074367982B70431C3E89428
:10033000F0400374F0F8E8C4540F28F87984B70348
:1003400002615EC313C3138721200802C313200A6E
:1003500006C3C898F8615E28F8500374FFF8882235
:10036000306915E5222408F52250037522FFC3E504
:1003700022955E4003855E227882B6041885222489
:10038000A824C3E524955E4002A85EC3E8956040BA
:1003900002A8608825C3E52594404002D26420CF9E
:1003A0000CD0E0D0D0C2D343E610D2AD32C2CF7869
:1003B00001E52960053074021529C3E5599401400F
:1003C00005755C0061D7755D00756400E55C24010E
:1003D000F55C5003755CFFD0E0D0D0C2D343E6108B
:1003E000D2AD32C0D0C0E0C2AF53917F53E67FC2DE
:1003F00060759100C3E49550F594E49551F59575B9
:100400009104D0E0D0D0D2AF32C2AF53E6EFC2AD4C
:10041000C0D0C0E0C0F0D2D3D2AFA8FBA9FCC2D8F4
:10042000307102817053DACF207E0343DA10307EC0
:100430000343DA20D271E580307E01F420E50281A9
:100440004788268927C1AC53DACF207E0343DA20C0
:10045000307E0343DA10C2D8C271307402C198787A
:1004600000E580307E01F430E502C1988859C17FF3
:0F04700053DACF207E0343DA20307E0343DA10C5
:10047F00C271206102A14053DACF207E0343DA100C
:10048F00307E0343DA20C2D8D27188548955C3E82D
:10049F009552F8E99553F9E4FB7E027A00C3E8948C
:1004AF008CE994005005755800A130C3E894C8E951
:1004BF0094005008E4D2E4FB7A0AA10DC3E89468D3
:1004CF00E994015008E4D2E3FB7A0FA10DC3E8943D
:1004DF00D0E994025008E4D2E2FB7A1EA10DC3E8E2
:1004EF0094A0E994055008E4D2E1FB7A3CA10DC336
:1004FF00E89498E994085008E4D2E0FB7A787E00FB
:10050F00C3E89556FCE99557FD30E708ECF4240154
:10051F00FCEDF4FD755800C3EC9AED9E5003755831
:10052F000188568957A854A955885289537802C112
:10053F007FC3E89526F8E99527F9307C02C163302F
:10054F007B02C163307A02C15C207502A163E9FDB1
:10055F00E8FCA182E9C313F9E813F8307902C15C12
:10056F00E9C313F9E813F8307802C15CE9C313FD4E
:10057F00E813FC206126C3EC941CED94024002A109
:10058F0099ED7018C3EC94C850120528C3E5289450
:10059F000A5002C198755900D270C198E5286002BF
:1005AF0015287400207F0B7888E67896B4030278BC
:1005BF009EE624FAFEE43400FFC3EC9EFCED9FFDA3
:1005CF0092087888E6B40327A2085009207D20C23C
:1005DF00AFD27DA1EB307D17C2AFC27DC286C29173
:1005EF00C295C290C292C296206902D26BD2AFA2BC
:1005FF00085017E6B4030DECF42401FCEDF43400BD
:10060F00FD02061978007900C1637888E6B40315F6
:10061F00EC33FCED33FDC3EC940AFCED9400FD507C
:10062F00047C007D00C3EC94FFED9400400678FF3E
:10063F007900C163EC856FF0A4C5F0A2F733F879A8
:10064F0000400302067F78FF790002067FE9C3139B
:10065F00F9E813F8307C0EE9600278FFC3E813382D
:10066F00F8E43400F9C3E894FFE99400400278FFFE
:10067F008859D270206102C198741FF4552F4BF521
:10068F002FC274E42B7002D274752918307403755D
:10069F00290A306102C1AC20740353DAFE752A06B1
:1006AF00307403752A0AD0F0D0E0D0D0C2D3D2ADC7
:1006BF0043E6103279010206E179030206E1790A75
:1006CF000206E1791E0206E179640206E179C802A9
:1006DF0006E17817E4D5E0FDD8FAD9F6227A147B33
:1006EF00780207087A107B8C0207087A0D7BB40218
:1006FF0007087A0B7BC8020708AC2575250179021C
:10070F00B27DE4C292D5E0FDE5256002D291D5E03D
:10071F00FDC291D5E0FDD292D5E0FDE525600A201E
:10072F007D02D286307D02D295E570D5E0FD207D29
:10073F0002C286307D02C2957496D5E0FDD9C1EA1A
:10074F00F8D5E0FDD8FBDBB1C2928C2522C37C002B
:10075F007D0075F00005F0EA33FAEB33FB50F6EB52
:10076F0013FBEA13FAC3E9FFE8FEE89AF8E99BF9ED
:10077F005004EFF9EEF8B3EC33FCED33FDD5F0DFB9
:10078F00EDF9ECF822E889F08A20D2D4F8A9F07BB1
:10079F000030F70B7BFFF42401F8E9F43400F9E89B
:1007AF008520F0A4ADF0F8E98520F0A4AFF0FEEDC0
:1007BF002EF974003FFA7C04C3EA13FAE913F9E83F
:1007CF0013F8DCF48BF030F70AE8F42401F8E9F4BD
:1007DF003400F9E889F0C2D4F8A9F0227882B6047F
:1007EF0003020848C3E5599401400302081085220B
:1007FF0024E4F53EF53FF540F541F542F547020893
:10080F00487882E6FC754701E522F523783879C7E9
:10081F00AA3AAB3BC3EB13FBEA13FAEC146013C316
:10082F00EB13FBEA13FAEC14146007C3EB13FBEAA8
:10083F0013FA12075C883E893F22E5476034C3E50F
:10084F003E9523F8E53F9400F9500CC3E89480E9F6
:10085F0094FF401602087DC3E8947FE9940050038B
:0E086F0002087D787F790002087D788079FF8D
:10087D008843894422E5476058E5432540F8E5441F
:10088D003541F9854420E4300701F43542FA30E76B
:10089D0009C3EA94F040150208BFC3EA940F500350
:1008AD000208BF78FF79FF7A0F0208BF7800790040
:1008BD007AF0C3E524955E5006E524600901D8E57C
:1008CD004420E70D01D8E54430E706884089418A88
:1008DD004222E547700302094378A1E6FAC3E543D6
:1008ED0033F8E54433F9120794E930E70BC3E89484
:1008FD0080E994FF4013211AC3E8947FE9940050D6
:10090D0002211A787F7900211A788079FFE820E793
:10091D0015C3E52398F84009C3E894014003020983
:10092D00417801020941E8F424012523F84003022E
:10093D00094178FF884522E54770030209A678A290
:10094D00E6FAA841A942120794E930E70CC3E894EE
:10095D0001E994FF401602097DC3E894FFE9940074
:10096D00500302097D78FF790002097D780179FF36
:10097D00E920E715C3E54598F84009C3E89401401F
:10098D00030209A478000209A4E8F424012545F81E
:10099D0040030209A478FF88242278FFC264E52D64
:1009AD005406702FD264C3E53B940A4009C3E52574
:1009BD0094405002C264E53B601974FF853BF0849E
:1009CD008537F0A4F8C5F0600278FFC3E895615053
:1009DD0002A8618860227883E6F520120F5175E830
:1009ED00901206C375E890E5E820ECFBA8BDA9BE02
:1009FD00120FFF756B55756C00C3740013FD7455A4
:100A0D0013FC74552CFC74003DFDECFAEDFBC3E8B2
:100A1D009AE99B4014E56B2455F56BE56C3400F5B4
:100A2D006CEA2CFAEB3DFB80E5AE6BAF6CC3E56C6D
:100A3D0013F9E56B13F8C3E913F9E813F8E56B281F
:100A4D00F569E56C39F56A7A03C3E913F9E813F82A
:100A5D00DAF7AA201A7009756B00756C00020A7D11
:100A6D001AEA6008EE28FEEF39FFDAF88E6B8F6C0C
:100A7D002275E890227883E6FFE5E820ECF7A8BD23
:100A8D00A9BE056DC3E56D94084052756D00E9FA78
:100A9D0079A0E76044EA7007E56E601B020AB8C3EF
:100AAD00E8956E6010E56E5006600C14020AC404E1
:100ABD0060F9020AC4E56EF56EC3946D401B755E58
:100ACD00C0C394044013755E80C39404400B755EDF
:100ADD0040C394044003755E0075BB0B22EFC394B5
:100AED0001601BC3E894FFE994035012C3E8956BB2
:100AFD00E9956C5009E55E601A155E020B20E55E06
:100B0D00F46010055E7888E6B40308E55E240440C1
:100B1D0002F55EA85EC3E524985002A824C3E895AB
:100B2D005F400AA85FE55FF46003855F5E7982B779
:100B3D000402614BC3E895604002A8608825E56D0D
:100B4D00B4070375BB1022743279A387F0A4C5F0E6
:100B5D00A2F733F8C3E8955E4002A85E8822882488
:100B6D008825886122753A00753B7F2275C820A8BB
:100B7D00CCA9CD75C824AA38AB3988388939C3E8D2
:100B8D009AF8E99BF9AA3AAB3BAC3AAD3B7E047FB0
:100B9D0002C3EB940440021E1FC3EB940840021ED7
:100BAD001FC3ED13FDEC13FCDEF7C3EA9CFAEB9DBE
:100BBD00FBEF6009C3E913F9E813F8DFF7EA28FA48
:100BCD00EB39FB8A3A8B3B400122753AFF753BFFAF
:100BDD002230600261DE854C50854D51D26043E676
:100BED0080227892E6FFC3E535948240010FC3E57C
:100BFD003594A040010FC3EF940640027F057E029D
:100C0D001E3072010EC3E53B940350060E0E30727A
:100C1D00010EC3E53B940250060E0E3072010EA973
:100C2D003BA83A7A04C3E913F9E813F8DAF7C3E8F5
:100C3D009EF8E99400F94009C3E89402E994005044
:100C4D00047802E4F9E9FBE8FAC3E913FDE813FCC3
:100C5D00884C894DC3EF94036037EF20E00DE82CED
:0F0C6D00F8E93DF9ECFAEDFB020C8BE828F8E909
:100C7C0039F9C3E89402F8E99400F97A02E4FBC369
:100C8C00EF9403400D8A4E8B4F884889498C4A8DCE
:100C9C004B22884E894F8A488B498C4A8D4B223087
:100CAC00600281ABD26043E680E52D54066027A834
:100CBC003AA93BE53494085006E820E002A94D75AA
:100CCC009100C3E498F594E499F595759104D2607C
:100CDC0053917F43E68022D265753D00752000025A
:100CEC000CF6D265753D00752040E52D540660026A
:100CFC00C265D2AF206005E53D60012278017A0221
:100D0C00C3E53B940540027802C3E53B940A4002DC
:100D1C007803C3E53B940F40027A03306904781ED4
:100D2C007A01206007E53D6003D2AF22D2AF00000C
:100D3C00C2AFC3E53BFB940F40027B0FEB04307357
:100D4C00012320620123F93069027982E58BC39972
:100D5C0040D0053DEAFBE59BF45440B52004DBF69E
:100D6C00A19220650281F6C265759100AE3AAF3B47
:100D7C00C3E49EF594E49FF595759104D26053916C
:100D8C007F43E68081F630650281F6D895D2AF229A
:100D9C0030690B0534206016753400020DBA2060E2
:100DAC000D20650A206B07158115810215FD22A8FF
:100DBC004EA94F75910053917FC3E498F594E49933
:100DCC00F595759104854850854951D26043E6806C
:100DDC002278003064053065027801E53575F0073E
:100DEC00A4F9E5F028F5F0E9A2F013A2F113A2F2B0
:100DFC0013F535C394785003753578C3E5359536BE
:100E0C004008D266C286C291C295306002C1168576
:100E1C004A50854B51D26043E68022C2AFC290C289
:100E2C0092C29630720B9001FC740ED5E0FD020E4E
:100E3C0065E53B54F86022E525600A207D02D286E8
:100E4C00307D02D2957401D5E0FD207D02C2863042
:100E5C007D02C295741AD5E0FD207D02D290307DC2
:100E6C0002D296759F56753C02020FE4C2AF207DEC
:100E7C0002C295307D02C2863072179001D9C2929F
:100E8C00207D02C296307D02C290740ED5E0FD0228
:100E9C000EA190013C306206E5256002D291207DC6
:100EAC0003759F76307D03759F36753C03020FE406
:100EBC00C2AFC290C292C29630720B9001B6740E41
:100ECC00D5E0FD020EFAE53B54F86022E525600AF8
:100EDC00207D02D295307D02D2867401D5E0FD20B2
:100EEC007D02C295307D02C286741AD5E0FD207D4C
:100EFC0002D296307D02D290207D03759F36307DD4
:100F0C0003759F76753C04020FE4C2AFC291307238
:100F1C0017900193207D02C290307D02C296C2923E
:100F2C00740ED5E0FD020F3790012A30620EE525D4
:100F3C00600A207D02D286307D02D295759F56754F
:100F4C003C05020FE4C2AFC290C292C29630720B43
:100F5C00900168740ED5E0FD020F7FE53B54F860FC
:100F6C0012E5256002D2917401D5E0FDC291741A8C
:100F7C00D5E0FDD292207D03759F76307D03759F61
:100F8C0036753C06020FE4C2AF207D02C286307D6E
:100F9C0002C29530721F900227207D02C290307DD4
:100FAC0002C296207D02C296307D02C290740ED58C
:100FBC00E0FD020FC490014E30620EE525600A2060
:100FCC007D02D295307D02D286207D03759F36300E
:100FDC007D03759F76753C01306B13120FFF740EF9
:100FEC00D5E0FD741AD5E0FDD290D292D296C266AD
:100FFC00D2AF22900128C286C291C295C290C292F1
:10100C00C296C262227880760908760908760408AE
:10101C0076010876030876FF08760A0876010876CA
:10102C0001087601788C76010876FF0876FF087641
:10103C00FF0876FF0876FF0876030876FF0876FF30
:10104C000876FF0876250876D008762808765008AA
:10105C0076040876FF08760208760008767A087619
:0F106C00FF087601227887E6FFC2727888E6C314
:10107B0094036008C27DE630E102D27DC27E78899E
:10108B00E630E102D27EC3EF94026008758E01D286
:10109B00730210A4758E00C273227880E614900040
:1010AB00809378A1F67881E6149000809378A2F66D
:1010BB00120FFF227886E61490008D9378A3F61218
:1010CB000FFF2222789CE67536FF75370CB40206AB
:1010DB007536A075370AB403067536827537052247
:1010EB00227896E6FA7897E6FB307F047A007BFF4E
:1010FB00C3EB9AFCC3948250027C82756F00056F20
:10110B00EC856FF0A4C3E5F0948040F222D27F11FE
:10111B00EC1206D27A007B007C101206C8E5592A25
:10112B00FA74003BFBDCF37C04C3EB13FBEA13FA0E
:10113B00DCF7FEC27F11EC22E5EF20E60375200001
:10114B000520903FFFE520146006901DFF14600002
:10115B009304600375EF12C2D353D9BF7581C0439B
:10116B00FF801206C375EF0243B203E5B3240420DC
:10117B00E702F5B3120FFF7580BF75A44075F17FC1
:10118B0075D4DF75909875A56775F26775D5007581
:10119B00A60175E241111112162E78988670C2AF16
:1011AB001206DC1206EC1206D21206F31206D2124B
:1011BB0006FA1206D2C2AFE4F8F6D8FD78C879C8A1
:1011CB00308507D9FBD8F7021C00111112162E110E
:1011DB007111A511BF11CE11CF11EB11EC789886BF
:1011EB0070120FFF75885075891275C8247591049C
:1011FB0075D84075A82275B80275E690759B8075F9
:10120B009D0075D10E75BC5875BB0B75BA1175E881
:10121B00801206C3D2AF1209E343DA01C2D8C271FE
:10122B001206DC753001D2617B037A0CE55870062F
:10123B007A0CDB0221C01206D220700221C0C270D0
:10124B00E559C3940240E3E52F541F855B5AF55BC8
:10125B00B55AD7DAD7C26153DACF207E0343DA20EF
:10126B00307E0343DA10C2D8C271C27575280012E2
:10127B0006D7307409C3E528940A4002D2751206CA
:10128B00C878023074027800C3E5599840F0C2AFB9
:10129B001206EC1206EC1206ECD2AF1206DC754607
:1012AB00007888E6B4030261881206C8788CE6C31E
:1012BB0094015003021388E530C3940150030213C9
:1012CB0088207435C3E55994FF5003021388C2AFCD
:1012DB00120701D2AF1206D7C3E559940150EFC2E2
:1012EB00AF1206EC1206CD1206ECD2AF1206D7C324
:1012FB00E55994FF40E90217D57F02D27F11EC121A
:10130B0006D7C2AFC27F11ECAE59C3E559947FD259
:10131B00AF40741206C3C2AF120701D2AFDFDC318C
:10132B0018C3EE94057897F61206DC12166F121797
:10133B00587F0AD27F11EC1206D7C2AFC27F11ECD5
:10134B00AE59C3E559947FD2AF50E61206C3C2AF74
:10135B001206EC1206CD1206ECD2AFDFD63118EE28
:10136B0024057896F61206DC12166F1217871206F2
:10137B00D711ECC3E55994FF40F40217D5C3E559D7
:10138B00954640038559461206D778017988E7B40C
:10139B0003027805C3E55998400241ACC2AF12076E
:1013AB0001120701120701D2AF1206DC753000E4FF
:1013BB00F531F5320531E531F470390532789AE6BD
:1013CB007819146012783214600D787D14600878E7
:1013DB00FA146003753200C3E53298401715327565
:1013EB0031B478998670C2AF120701D2AF78988664
:1013FB00701206D71206CDE529700530740221C094
:10140B0078012074027806C3E5599840A77888E6DE
:10141B00C3940360031206D7E529700221C0C2AF43
:10142B00120FFFE4F522F523F524F525D2AF7885CD
:10143B008662F53EF53FF540F541F542F56DF54712
:10144B00F52CF52DF535120B72756D0875BB101259
:10145B0006C3120A7EE5E820ECFBA8BDA9BEE97025
:0F146B0001F8886E120A82756D0875BB107887BC
:10147A00E6FE760211717887EEF6C2AF755EFF124C
:10148A000B5485225E85225F852260D2AF752201C8
:10149A00752401752501855D64756501D268D26977
:1014AA00753400120F51120F93120B72120B79122C
:1014BA000BEF0214CA120FFF1171756D0075BB0B89
:1014CA00120CEE120D9C120DBB1207EB120DDD125F
:1014DA000E27120B79120BDE120BEF120CAB120C49
:1014EA00E3120D9C120DBB1208491209A7120DDD59
:1014FA00120E78120B79120BDE120BEF120CAB12D2
:10150A000CEE120D9C120DBB120882120DDD120E8A
:10151A00BC120B79120BDE120BEF120CAB120CE39E
:10152A00120D9C120DBB1208DF120DDD120F1612DE
:10153A000B79120BDE120BEF120CAB120CEE120D22
:10154A009C120DBB120944120DDD120F51120B79B8
:10155A00120BDE120BEF120CAB120CE3120A7E1204
:10156A000D9C120DBB120A82120DDD120F93120B83
:10157A0079120BDE120BEF120CAB306938206B3587
:10158A0085615E85615F855D6475650179327A0A78
:10159A00C3E534994012C269D26A8A3385615E759D
:1015AA005FFF7560200215BFC3E55994014003022D
:1015BA0014CA0215FD306A1E206B1BE5331470072E
:1015CA00C26A755EFF81BFF533C3E55994014003D2
:1015DA000214CA0215FDC3E55C94FA50163074046D
:1015EA00E529600FC3E53B78F0306B0278609850CC
:1015FA000281CAC2AF120FFF7887E6FE7602117126
:10160A007887EEF6E4F522F523F524F525F562C28E
:10161A0068D2AF1206C3120FFF307406E5297002B2
:10162A0021C061BA901A0D78201216B1E520B4557E
:10163A000CA31216B1E520B4AA0302164F11111217
:10164A00166F02166E901A0378807B0A1216B1A3DF
:10165A0008DBF9901A0F788C7B151216B1A308DBF8
:10166A00F9901A2422C2AF1216F01216CA901A0062
:10167A00740D1216B6A374021216B6A374131216B8
:10168A00B6901A0378807B0A1216B5A308DBF99084
:10169A001A0F788C7B151216B5A308DBF9121703FB
:1016AA001216E1901A2422E493F622E6438F01539C
:1016BA008FFD75EF0275B7A575B7F1F0538FFE224E
:1016CA00438F02438F0175EF0275B7A575B7F19085
:1016DA001A0DF0538FFC22901A0D7455D1B6901A38
:1016EA000E74AAD1B6227A3079D07820901A40D1D5
:1016FA00B1E520F709A3DAF7227A3079D0901A40B7
:10170A00E7D1B609A3DAF922AB71A872BB01027953
:10171A0080BB02027981BB03027982BB040279840D
:10172A00BB05027983BB06027986BB07027992BBA5
:10173A0008027987BB0902799CBB0A027988BB0B2C
:10174A00027989E8F7227C051206DCDCFB22C2AFAB
:10175A001206EC1206F31206FA1207011206CD124D
:10176A0006EC1206F31206FA1207011206CD120649
:10177A00EC1206F31206FA120701D2AF22C2AF1216
:10178A0007011206FA1206F31206EC1206CD120728
:10179A00011206FA1206F31206EC1206CD1207011E
:1017AA001206FA1206F31206ECD2AF22AE71AF722B
:1017BA00C2AF1206EC1206EC1206EC1206CDDEF2ED
:1017CA001207011206CDDFF8D2AF22F158F150F11B
:1017DA0050757101757201757300F1B67C05AD59CA
:1017EA001206DCC3ED955970F5C3E5599401400A18
:1017FA00C3E55994FF403702181512171212166FD3
:10180A00121758C2AF75EF12121750DCD10573C305
:10181A00E5739403500280C21217500572E57114E1
:10182A0090009A93F808C3E57298500280A912179B
:10183A00501217500571C3E571940C50028095122D
:0D184A00101112166FC2AF75EF1212175079
:101A00000D02130909040103FF0A01010155AA018E
:101A1000FFFFFFFFFF03FFFFFF25D0285004FF0259
:051A2000007AFF01FF48
:101A400023416C69676E424C3135502320202020A1
:101A500023424C48454C4923463333302320202031
:101A60002020202020202020202020202020202076
:101C0000C2AFC2D353D9BF7581C043B20343FF8073
:101C1000752438752503B1BF75EF0275E24043F1B5
:101C20002053A4DFD285780379E67C1075220075F5
:101C30002300901DCC7B0675249875250130850204
:101C4000813D208508D8FBD9F9DCF781AD308508C6
:101C5000D8FBD9F9DCF781ADB17FE493A3C39A60D7
:101C6000028126DBDDB171600281267B08E493FAF4
:101C7000A3B152DBF87A30B152752200752300B15E
:101C800071EAFCEBFDC3ED94FE400EB1718A278B27
:101C900028ED30E0048A828B83B1717AC270D8C398
:101CA000ED94FE601050CEBD0022EC600675200061
:101CB0000200008100A827A9280809D804D90281B8
:101CC000C9B175EA89AAF281BB0D8199C3ED94036C
:101CD0005049EDA2E092007AC5C3E5829400E58305
:101CE000941C5093200010438F02438F0175B7A5B9
:101CF00075B7F1F030001FA827A9280809438F0104
:101D0000538FFDD804D902A11689AAE275B7A5752B
:101D1000B7F1F0A3A103538FFC81757AC1BD030C09
:101D2000E493A3FAB136DCF8B12E81758177AA224B
:101D3000AB23B152EBFAEA6222752608C3E52313FE
:101D4000F523E52213F52250066323A0632201D573
:101D500026EAB1BFB1BF75260AEAF4200102D28596
:101D6000300102C285B1BFC3134002C201D526EBC8
:101D700022B175EAFB208502A175308502A17A7532
:101D80002608AE24AF25C3EF13FFEE13FEB1C3B197
:101D9000BFC3EA133085024480FA30E703632201AF
:101DA000C3E52313F523E52213F52250066323A090
:101DB000632201D526D9E52265236523F52222AECB
:101DC00024AF250E0FDEFEDFFCD20122424C486517
:0A1DD0006C6934373132F33006013C
:00000001FF
